:100000000C941C040C9454040C9454040C94540448
:100010000C9454040C9454040C9454040C94540400
:100020000C9454040C9454040C94B5160C944B1B6F
:100030000C9426260C9454040C9454040C945404EC
:100040000C9454040C9454040C9454040C945404D0
:100050000C9454040C948E170C9454040C94540473
:100060000C9454040C9454040C9454040C945404B0
:100070000C9454040C9454040C9454040C945404A0
:100080000C9454040C9454040C9454040C94540490
:100090000C9454040C9454040C9454040C94540480
:1000A0000C9454040C9454040C9454040501090257
:1000B000A10185020901A1000509190129081500FE
:1000C0002501950875018102050109300931158165
:1000D000257F95027508810609381581257F9501D0
:1000E00075088106050C0A38021581257F95017572
:1000F000088106C0C005010980A101850319012AF4
:10010000B700150126B700950175108100C0050CD8
:100110000901A101850419012AA002150126A002E6
:10012000950175108100C005010906A1018506052C
:100130000719E029E71500250195087501810205D9
:1001400007190029EF1500250195F07501810205B9
:10015000081901290595057501910295017503910D
:1001600001C00660FF0961A1010962150026FF00B8
:100170009520750881020963150026FF00952075FA
:10018000089102C005010906A101050719E029E748
:1001900015002501950875018102950175088101F9
:1001A0000507190029FF150026FF0095067508812F
:1001B000000508190129059505750191029501753C
:1001C000039101C0000000000000000000000000DA
:1001D000000000000000000000000000000000001F
:1001E00000000000000000007E0F00D4FFFFFFC7EA
:1001F0000000007800000000000000002A2B28000A
:1002000000000000000000000000000000000029C5
:10021000000000002C1E3420212224342627252E05
:10022000362D3738271E1F2021222324252633333D
:10023000362E37381F0405060708090A0B0C0D0E69
:100240000F101112131415161718191A1B1C1D2F35
:100250003130232D350405060708090A0B0C0D0E55
:100260000F101112131415161718191A1B1C1D2F15
:100270003130354C0001010101010101010102028F
:100280000202020202020203030303030303030444
:10029000040404040404050505050506060606060F
:1002A000070707070708080808090909090A0A0AC9
:1002B0000B0B0B0C0C0C0D0D0D0E0E0E0F0F0F106B
:1002C00010111111121213131414151516161717F5
:1002D000181819191A1A1B1B1C1D1D1E1E1F202061
:1002E000212222232424252626272829292A2B2CAB
:1002F0002D2D2E2F30313232333435363738393ACE
:100300003B3C3D3E3F404142434445464748494AC5
:100310004C4D4E4F50515354555658595A5B5D5E93
:100320005F616264656668696B6C6D6F707273752E
:1003300077787A7B7D7E8082838587888A8C8E8F92
:1003400091939596989A9C9EA0A2A3A5A7A9ABADC0
:10035000AFB1B3B5B7BABCBEC0C2C4C6C9CBCDCFAE
:10036000D1D4D6D8DBDDDFE2E4E7E9EBEEF0F3F55C
:10037000F8FAFDFF002636460027374700283848A0
:1003800000293949002A3A4A002B3B4B01263646C0
:10039000012737470128384801293949012A3A4AB3
:1003A000012B3B4B022636460227374702283848A6
:1003B0000074645400756555007666560079695975
:1003C000007A6A5A007B6B5B01756555017666564B
:1003D00001796959017A6A5A017B6B5B0274645432
:1003E000027565550276665600A4948400A595852D
:1003F00000A6968600A7978700A8988800A99989E3
:1004000001A4948401A5958501A6968601A79787E6
:1004100001A8988801A9998902796959027A6A5ACA
:10042000027B6B5B002E3E4E002F3F4F0030405052
:1004300000314151003242520033435301AC9C8C95
:10044000012E3E4E012F3F4F0130405001314151AE
:10045000013242520133435302A7978702A898887A
:10046000007C6C5C007D6D5D007E6E5E0081716164
:10047000008272620083736301AD9D8D017C6C5CB0
:10048000017D6D5D017E6E5E01817161018272622E
:100490000183736302A9998900AC9C8C00AD9D8D8A
:1004A00000AE9E8E00AF9F8F00B0A09000B1A191D2
:1004B00001AE9E8E01AF9F8F01B0A09001B1A191BE
:1004C00002293949022A3A4A022B3B4B29003A00B9
:1004D0003B003C003D003E003F0040004100420028
:1004E0004300440045004C00460035001E001F003C
:1004F0002000210022000000230024002500260007
:1005000027002D002E002A002B0014001A000800DE
:10051000150017001C0018000C00120013002F001B
:10052000300031004B0039000400160007000900BC
:100530000A002A000B000D000E000F0033003400EB
:1005400028004E00E1001D001B00060019000500F8
:10055000280011001000360037003800E500520076
:100560000000E000E300E20000002C00E000E100F9
:100570002C000000E6000151E400500051004F0043
:10058000005C010001000100010001000100010008
:100590000100B200B300AF00B100145CDE5C0100EA
:1005A0000100010001000100010000000100010044
:1005B000010001000100010001005300C25CC35CA6
:1005C000C95CC55C010001000100010001000100DF
:1005D00001000100010001004A000100CC5CCA5C7E
:1005E000CB5C0100010001000100010001000100DD
:1005F0000100010001004D000100010001000100A7
:1006000001000100010001000100010001000100E2
:10061000A800A90000000100010001000000010085
:10062000010001000100000001000100AE00AC006B
:10063000AA00AB000100010001000100010001005F
:1006400001000100010001000100010001000100A2
:100650000100010001000100010001000100000093
:100660000100010001000100010001000100010082
:100670000100010001000100010001000100010072
:100680000100010001000100010001000100010062
:100690000100010001000100010001000100010052
:1006A0000100010001000100010001000100010042
:1006B0000100010001000100010001000100010032
:1006C0000100010001000100000001000100010023
:1006D0000000010001000100010000000100010014
:1006E0000100010001000100010001000100010002
:1006F00001000100010001000100010001000100F2
:1007000001000100010001000100010001000100E1
:1007100001000000010001000100010001000100D2
:1007200001000100010001000100010001000100C1
:1007300001000100010001000100010001000100B1
:1007400001000100010001000100010001000100A1
:100750000100010001000100010001000100010091
:100760000100010001000100010001000100010081
:100770000100010001000100010001000000010072
:100780000100010000000100010001000100000063
:1007900001000100010001000100010009025B00ED
:1007A000030100A0FA09040000010301010009216E
:1007B000110100012240000705810308000109041E
:1007C00001000203000000092111010001222200A2
:1007D0000705820320000107050303200001090427
:1007E0000200010300000009211101000122B600EE
:1007F00007058403200001120100020000000842E6
:1008000058504B01000102000118034B004E0049F3
:10081000004700480054005F0050004C0055005352
:100820000000000E0358002D0042004F00570053F7
:10083000000000040309040011241FBECFEFDAE01A
:10084000DEBFCDBF04B603FE18C08091570690915D
:100850005806A0915906B0915A068730904BA74090
:10086000B04B59F410925706109258061092590640
:1008700010925A06E0E0F8E3099526E0A8EDB2E010
:1008800001C01D92A735B207E1F712E0A0E0B1E088
:10089000E8E8FCE502C005900D92A83DB107D9F744
:1008A0000E944D260C94072E0C940000E8EDF0E019
:1008B00080818E7F80831092E2001092DA00109285
:1008C000E100A0EEB0E08C9181608C9380818F7705
:1008D000808319BCA7EDB0E08C918E7F8C938081D2
:1008E0008F7E80831092F10508952091E40030916D
:1008F000E50095E6A9012091EC00822F817020FF90
:1009000006C08091E80080FF06C080E00895209135
:10091000E80022FD1AC080911606882389F08530F0
:1009200089F08091EB0085FD0FC02091E4003091AB
:10093000E50042175307F9F29150E1F684E008957B
:1009400082E0089583E0089581E00895EF92FF9298
:100950000F931F93CF937C018B010E947504C82FC6
:10096000811117C08091E80085FD0BC08091E800DF
:100970008E778093E8000E947504882399F3C82F2E
:1009800008C0F70181917F018093F10001501109A6
:1009900049F78C2FCF911F910F91FF90EF90089501
:1009A0008091180687FF13C08091E80082FF06C07F
:1009B0008091E8008B778093E80004C08091160650
:1009C0008111F2CF0895809116068823D9F3809182
:1009D000E80080FFF8CF8091E8008E77ECCF982F69
:1009E0009093E900242F762F50E0891731F0709111
:1009F000EC002091ED005091F00021FD07C09F5FB9
:100A0000973071F78093E90081E008953091EB0011
:100A10003E7F3093EB003091ED003D7F3093ED0051
:100A20003091EB0031603093EB007093EC00209339
:100A3000ED005093F0002091EE0027FDE0CF80E024
:100A40000895B0E0A0E0E7E2F5E00C946D2CC8ED6D
:100A5000D0E088818F7E8883E7EDF0E0808181603F
:100A6000808384E082BF81E08093F10588818E7F5E
:100A7000888302EE10E0F80110821092DA0081EE15
:100A8000C82ED12CF601108288818F7788838881C7
:100A90008068888388818F7D888319BC10921606B0
:100AA00010921706109215061092140690EEE92E79
:100AB000F12CF70180818B7F80838881816088831E
:100AC00042E060E080E00E94EF04F60180818E7FCA
:100AD0008083F80180818160808380818860808349
:100AE000F70180818E7F8083888180618883CDB784
:100AF000DEB7E8E00C94892CFC0180911E069091F1
:100B00001F0686179707A0F06115710529F49091CB
:100B1000E8009E779093E80090E06115710551F42C
:100B2000911108C08091E80082FF34C080E00895F0
:100B3000BC01F2CF809116068823C1F18530C1F146
:100B40008091E80083FD30C08091E80082FDEACF0B
:100B50008091E80080FFE1CF8091F3002091F200C6
:100B6000382F6115710519F02830310558F091E0E2
:100B70002830310509F090E02091E8002E7720938D
:100B8000E800CBCF81918093F100615071092F5F14
:100B90003F4FE7CF80911606882341F0853041F022
:100BA0008091E80083FFBECF81E0089582E0089540
:100BB00083E0089508958091F3050895209113012D
:100BC0002223C9F02091EC0527FF15C0E62FE695FA
:100BD000E695E695EE31D8F4E80FF92FF11D677030
:100BE00021E030E001C0220F6A95EAF7209582816A
:100BF000282322830895FC013296089621916213DE
:100C000003C0DF0111971C92E817F907B9F708959F
:100C1000209113012223C1F02091EC0527FF14C07D
:100C2000E62FE695E695E695EE31F8F4E80FF92F14
:100C3000F11D677021E030E001C0220F6A95EAF7EC
:100C40008281822B82830895FC0132962FEF30E05F
:100C50004191641751F02F3F19F4411101C0232F26
:100C60003F5F3630A9F72F3F09F40895820F911D99
:100C700027FD9A95FC01628308952091E505309146
:100C8000E6052817390771F09093E6058093E5058E
:100C9000E091E305F091E405309721F00084F185BF
:100CA000E02D099508952091E1053091E20528177E
:100CB000390771F09093E2058093E105E091E30537
:100CC000F091E405309721F00680F781E02D099539
:100CD0000895E091E305F091E405309729F0019043
:100CE000F081E02D0995089580E00895FA018111C1
:100CF00001C0FB0109950895E4E2F6E0248130E1AA
:100D0000231B08F420E024838091E003816080931A
:100D1000E0030895E4E2F6E0248130E1230F08F4D3
:100D20002FEF24838091E00381608093E003089596
:100D300090912406937071F08093250660932606A7
:100D4000493C08F048EC409327068091E003822B51
:100D50008093E0030895E4E2F6E0438120E1421B42
:100D600008F440E0818121E0628190E00E949806D1
:100D70000895E4E2F6E0438120E1420F08F44FEFEA
:100D8000818121E0628190E00E9498060895E4E26A
:100D9000F6E0628120E1621B08F460E0818121E0DD
:100DA000438190E00E9498060895E4E2F6E06281B3
:100DB00020E1620F08F46FEF818121E0438190E030
:100DC0000E9498060895E4E2F6E0818121E04381E3
:100DD00062818850990B0E9498060895E4E2F6E03B
:100DE000818190E021E04381628108960E9498060B
:100DF000089590912406937061F081110BC0946066
:100E000090932406109212018091E003862B809328
:100E1000E0030895823110F09464F2CF880F880FB8
:100E2000982BEECF8091240686958695815009F403
:100E300081E161E00E94F90608958091240686957B
:100E400086958F5F823108F081E061E00E94F906AB
:100E50000895EF92FF920F939701201B31092F3FC6
:100E6000310519F010F02FEF30E02095382F320FB8
:100E700008F43FEF832F0F91FF90EF900895EF92CA
:100E8000FF920F939701201B31092F3F310519F075
:100E900010F02FEF30E0322F3095482F430F08F439
:100EA0004FEF842F620F0F91FF90EF900895EF9214
:100EB000FF920F931F930E0D1F2D111DF90137FF88
:100EC00003C0F195E195F10924E0EE0FFF1F2A958B
:100ED000E1F7EF3FF10519F014F0EFEFF0E09A01C0
:100EE00057FF03C031952195310994E0220F331F3C
:100EF0009A95E1F72E173F070CF4F901E00FF11F67
:100F0000EF3FF10519F010F0EFEFF0E0E095282F3A
:100F10003E2F230F08F42FEF822F1F910F91FF9088
:100F2000EF900895EF92FF920F93970195E0099F3C
:100F3000200D311D11242F3F310519F010F02FEF36
:100F400030E02095382F320F08F43FEF832F0F91B8
:100F5000FF90EF90089522E8241B08F420E0620F30
:100F600008954095282F429F412D1124842F0895E4
:100F7000EF920F93972F23E0029FB00111247595F4
:100F800067956E0D792F0F91EF900895E42FF0E0A3
:100F9000EE0FFF1FEA52FE4F6081621B0895E42F9F
:100FA000F0E0EE0FFF1FEB52FE4F6081621B0895D1
:100FB000622F08950E94FF1108950E94C1110895A3
:100FC0000F931F9310E0F801EE0FFF1FEB52FE4F3F
:100FD00090819C5597FD9195000F111FF801EA52E1
:100FE000FE4F00810152110B2003F001219FF00DF3
:100FF000112408E310E0091B110997FD1395400324
:101000009001419F300D1124E20FF31F9F01220F29
:10101000331F2E0F3F1F37FF02C021583F4F220FB3
:10102000232F221F330B620F1F910F910895FC0194
:101030009B01009729F480E077FF2BC080E808959A
:10104000AC0197FF04C044275527481B590BB90131
:10105000640F751F37FD10C0241B350BC901A5E0B7
:10106000880F991FAA95E1F70E949A2C80E2861BAF
:10107000F7FF0FC081950895CB0165E0880F991F98
:101080006A95E1F7BA01621B730B0E949A2C80E605
:10109000EECF0895EF920F93CF93DF93D72FC82F02
:1010A000C9010E19BA010E941708602F681B7D2F15
:1010B0008C2FDF91CF910F91EF900895EF920F93C6
:1010C0001F93CF93DF93D62FC72F182FC9010E1967
:1010D000010FBA010E941708081B202F219F212D04
:1010E0001124822F6D2F7C2FDF91CF911F910F91B3
:1010F000EF9008950F93CF93DF93D72FC82FC90197
:10110000BA010E941708682F600F7D2F8C2FDF9186
:10111000CF910F910895E82F86FDE0952E2F2F7027
:1011200086FD2F5FE695E695E695E670F0E0EC59D2
:10113000FE4F9181929F902D212D112492959F70A9
:101140002295207F922B2081920F87FD919580E838
:10115000890F0895AC018230910508F408959FEF3E
:10116000413E8EE1580740F49A0195E03695279567
:101170009A95E1F798E0920F61E0E62FE90FFF27DB
:10118000FF1F9F0135952795822F229FF001239FF6
:10119000F00DF00D11244E175F0738F49FEF920FFA
:1011A000961758F78FEF860F08952F3FE9F361E008
:1011B000620FF6CF30E020E0869F212D969F200D14
:1011C000311D1124C9010895AF92BF92CF92DF92D1
:1011D000FF920F931F93CF93DF93362F472FE82F64
:1011E000F0E0EC58FD4F71110FC0E4918E2F2E2FBF
:1011F0006E2F722FDF91CF911F910F91FF90DF9093
:10120000CF90BF90AF900895C72FD0E02491F22ED9
:10121000022F10E056E0659FC0011124EFEFF0E0CF
:10122000BF010E944F2C832F90E0880F991F35E556
:10123000369FD001379FB00D11248A1B9B0B982F2E
:10124000990F980F6F01CC1ADD0AC09ED001C19E84
:10125000B00DD09EB00D11248B2F499FA0011124F9
:10126000452F55276F01C41AD50AC09EA001C19E03
:10127000500DD09E500D11245F01A91AB108AC9EEB
:101280006001AD9ED00CBC9ED00C1124CD2CDD2471
:10129000EC19FD09E09FE001E19FD00DF09FD00D1A
:1012A0001124ED2F62307105A1F050F46115710524
:1012B00009F49ECF6130710581F0EB2F852F98CF17
:1012C0006430710569F080F06630710509F490CFE3
:1012D000F4CFE22F2B2F8D2F8BCFE22F252F88CF0E
:1012E000EB2F822F2D2F84CF2B2F8F2DE52F80CF0B
:1012F0002F923F925F926F927F928F929F92AF92C6
:10130000BF92CF92DF92EF92FF920F931F93CF93F2
:10131000DF93CDB7DEB72A970FB6F894DEBF0FBEC6
:10132000CDBF8B837E836D832091140182E1289F42
:10133000802D11248F838E5E89838A83873510F0F8
:1013400036E53A8380912A068C83FF81EF2FF0E007
:10135000FA87E987CF01880F991F9C012B523E4FD6
:1013600069013B81832F90E0FC013196F887EF8380
:101370008A8199859817E8F081E0E981E63508F0DF
:1013800080E02A960FB6F894DEBF0FBECDBFDF9186
:10139000CF911F910F91FF90EF90DF90CF90BF9072
:1013A000AF909F908F907F906F905F903F902F9025
:1013B0000895E985FA85EF57FD4F808190911501D9
:1013C0008923F1F020902506309026062F8138855C
:1013D000265D394F39015B8010E0FC815F16D0F04B
:1013E00020912706129F112D1124B101812F0E94F7
:1013F000E408462F282F672F89859A850E94DD07EC
:1014000029853A852F5F3F4F3A87298732E0C30EFF
:10141000D11CAECFF30181913F01F601A080A81A43
:10142000BB088180F3018781881A9908AA9C9001E2
:10143000AB9C300D300D1124889CC001899C900D0F
:10144000900D1124820F931F0E94AA08082F60910B
:10145000280621E0620F08F46FEFF301EE0FFF1F83
:10146000EA52F640858996890E94DA087C01940147
:10147000A501B101812FED81FE8109951B015394D6
:10148000182FABCFB0E0A0E0E8E4FAE00C946D2CAC
:101490008C01C091140182E1C89FC02D112422E16A
:1014A000D22EDC0ECD2C26E52D1510F496E5C92E96
:1014B0002091280631E0230F08F42FEF30E050E0B0
:1014C00040E06FEF7FEF80E090E00E94A42D790173
:1014D000D0E02C2FCC1550F081E0F5E5FD1508F497
:1014E00080E0CDB7DEB7E8E00C94892CFE01EF5721
:1014F000FD4F808190911501892311F140912A06B9
:101500004150042E000C550B47FF1CC0C7016091D1
:10151000280621E0620F08F46FEF0E94DA08AC01A0
:10152000609125067091260680912706F80109959D
:101530000E94E408462F282F672FCE010E94DD0766
:101540002196C7CFFA01E65DF94F818982130AC05F
:10155000FA01EE0FFF1FE65DF94F818D928D8E151A
:101560009F05A8F241505109CFCFB0E0A0E0EBEBCE
:10157000FAE00C94682C5C01C091140182E1C89FD0
:10158000C02D112412E11C0FF12E173510F036E595
:10159000F32E609128066695809120069091210691
:1015A0000E94DA08782ED0E0CF1548F081E0163599
:1015B00008F080E0CDB7DEB7EDE00C94842CFE019E
:1015C000EF57FD4F8081909115018923C9F1CE011C
:1015D000880F991F85589E4FFC01E65AFF4F2081C6
:1015E000422F4C55550B6A01855A9F4FFC01808153
:1015F000282F2152330B4901449F9001459F300D04
:10160000300D1124889CC001899C900D900D1124EF
:10161000820F931F0E94AA08082F609125067091DF
:10162000260680912706E72C9401A601F50109956D
:101630000E94E408462F282F672FCE010E94DD0765
:101640002196B2CFB0E0A0E0E8E2FBE00C946E2C73
:101650007C01C091140182E1C89FC02D112412E1C8
:101660001C0F012F173508F006E5609128066695D6
:10167000669521E0620F08F46FEF8091200690914B
:1016800021060E94DA08D82ED0E0C01748F081E089
:10169000163508F080E0CDB7DEB7E7E00C948A2C71
:1016A000FE01EF57FD4F808190911501892391F044
:1016B0006091250670912606809127062D2D4C2FCE
:1016C000F70109950E94E408462F282F672FCE01C5
:1016D0000E94DD072196D9CF4091AE03803F59F497
:1016E0008091AF0387FF0DC01092AF0341110BC073
:1016F0001092A60308C0813F81F48091AF031816B1
:101700009CF3442381F08091B0039091B103892B25
:1017100009F05AC01092A5030895823F49F447FF8B
:10172000F0CF1092AE038091AF038111ECCFE0CFE8
:10173000833F19F41416ACF3E4CF9091B003893FC2
:1017400029F41916F4F61092B003DBCF8A3F19F48E
:1017500097FFD7CFF8CF9091B1038B3F29F497FF34
:10176000D0CF1092B103CDCF8C3F19F41916CCF322
:10177000C8CF9CE0980F953090F4845F990B21E0DE
:1017800030E0B90102C0660F771F8A95E2F7CB01FE
:1017900080959091AD0389238093AD03B2CF8D3FA7
:1017A00031F48091A7038E7F8093A703AACF8E3F49
:1017B00021F48091A7038D7FF7CF8F3F09F0A1CF50
:1017C0008091A7038B7FF0CF08958091A70380FDC0
:1017D00016C081FD16C082FD16C08091A503882326
:1017E000A1F0883280F428E0829FC001112468E2D1
:1017F00070E00E949A2C862F672B39F0089582E0C2
:10180000089584E0089588E0089581E00895809126
:10181000A70380FD14C081FD14C082FD16C0809115
:10182000A603882381F08E3180F420E5829FC001D9
:1018300011246EE170E00E949A2C862F089584E1B5
:10184000089588E2089588E0089580E50895803F2E
:1018500031F40E94070C81958093AF030895813F76
:1018600019F40E94070CF8CF823F31F40E94070C54
:1018700081958093AE030895833F19F40E94070C6D
:10188000F8CF893F29F40E94E50B8093B0030895B7
:101890008A3F21F40E94E50B8195F7CF8B3F31F40D
:1018A0000E94E50B81958093B10308958C3F19F454
:1018B0000E94E50BF8CF9CE0980F953070F4845FA0
:1018C000990B21E030E001C0220F8A95EAF7809160
:1018D000AD03822B8093AD0308958D3F31F4809149
:1018E000A70381608093A70308958E3F21F4809120
:1018F000A7038260F7CF8F3FB9F78091A703846079
:10190000F1CF80E00895F894E82FE295EF70F0E0D1
:1019100031A1282F2F7081E090E001C0880F2A9517
:10192000EAF7982F9095932391A392A1892B82A3F4
:10193000789408959091EC0592FF06C0282F2871A5
:101940002830F9F4877F846093FF06C0282F287120
:101950002831F1F4877E84612091ED0520FF06C0D7
:10196000382F38713830D9F4877F816021FF06C065
:10197000282F28712831D1F4877E816194FD877EDC
:101980000895282F24712430F9F68B7F8860DCCFEE
:10199000282F2471243101F78B7E8861DDCF382F09
:1019A0003171313019F78E7F8860E0CF282F217197
:1019B000213121F78E7E8861E1CFCF93DF93EC0157
:1019C00082389105A9F1D8F58133910509F496C0C3
:1019D00048F58932910509F48AC08A9709F495C0BF
:1019E000C11521E5D20708F0BCC0C11530E5D30709
:1019F00008F014C1C83ED10508F09CC0C03ED10516
:101A000060F5C83AD10508F087C0C53AD10508F09D
:101A1000FDC0C130D10509F12097F9F0C430D105DE
:101A2000E0F440C08533910509F45AC0C997C1F666
:101A30008091EC05837089F0C0EED0E00EC0833E4B
:101A4000910599F170F4803E910501F1823E910576
:101A500039F68091EC0582FD21C0CE01DF91CF9156
:101A60000895863E910561F1873E910571F1843EAE
:101A7000910509F0B5CF8091ED0581FFEECF809102
:101A8000EC05C7EED0E084FD0DC0E7CF8091EC05FA
:101A900080FD12C19091ED0590FFDFCFC3EED0E045
:101AA00084FFDBCFD0E0C0E0D8CF8091EC0582FD91
:101AB00006C19091ED0590FDBFCF84FFCECFF2CF50
:101AC0008091EC0583FDDDCFC8CF8091EC0583FDCF
:101AD000F9C09091ED0591FFF0CFC4EED0E0BDCFFD
:101AE0008091EC0585FFB9CFC9E2D0E0B6CF8091F7
:101AF000EC0585FFB2CFC5E3D0E0AFCF8091EC0518
:101B000086FFABCFCAE2D0E0A8CF8091EC0586FF7C
:101B1000A4CFC1E3D0E0A1CFCF3BD10518F6C85A7E
:101B2000D0E0CC0FDD1FC35EDE4F0990D881C02D01
:101B3000D46493CFC11540E2D40758F4C11581E0B5
:101B4000D80708F08ACFC03FD10508F4ABCFD065E5
:101B500084CFC11590E4D90708F4A4CFDF70D06A10
:101B60007CCFC11525E5D20700F5C11534E5D307B3
:101B700008F08AC0C11543E5D40708F071C0C1154B
:101B800082E5D80708F467C0CE018370992721E069
:101B900030E002C0220F331F8A95E2F7C695C69542
:101BA00080E2C89FE001112452C0C11599E5D90710
:101BB000A8F4C11528E5D20708F06BC0C11536E5B9
:101BC000D30708F06FCF8C2F0E949A0CC82FD0E05B
:101BD000DC2FCC27CC27DF71D0623FCFC1154AE57F
:101BE000D40708F45BC0CE0190568115904208F0EE
:101BF00059CF8D2F8F710E949A0C90E0982F8827D3
:101C000088279F719C012C2BE901E6CFC55AD0E0B3
:101C1000C65EDE4FC881D0E0D0641FCFCE01E4E0C5
:101C200096958795EA95E1F783702C2F2695269552
:101C3000237040E2249F90011124382B8C2F837055
:101C4000C1E0D0E002C0CC0FDD1F8A95E2F7C22BC5
:101C5000D32BDC6802CFDC2FCC27C16FD06AFDCE3E
:101C6000CE018370992721E030E002C0220F331F9C
:101C70008A95E2F7C695C69590E2C99FE0011124C6
:101C8000C22BD32BDA68E9CEDC2FCC27C46FD06A05
:101C9000E4CEDC2FCC27C06FD06ADFCE8C2F8F70C4
:101CA0000E949A0C34E0D695C7953A95E1F7CF702B
:101CB0009C2FEC01D069D1CEC9E3D0E0CECEC2EEEC
:101CC000D0E0CBCEC6EED0E0C8CE80917A038111B1
:101CD00010927A03089580959091790398239093B8
:101CE000790308958091560390912503981301C0BC
:101CF00008958F5F8770FACF292F963078F58F304F
:101D000068F590E03FE0239F800D911D1124682F1E
:101D1000677023E0969587952A95E1F7FC01EE0F11
:101D2000FF1FE80FF91FE550FD4F50E040E080E055
:101D3000219130E0062E02C0369527950A94E2F7ED
:101D400021703327042E01C0220F0A94EAF7822B58
:101D50004F5F5F4F4330510559F7089580E0089574
:101D6000292F963098F58F3088F590E03FE0239F3B
:101D7000800D911D1124282F277041E001C0440FD0
:101D80002A95EAF723E0969587952A95E1F7FC01D5
:101D9000EE0FFF1FE80FF91FE550FD4F30E020E088
:101DA00070E05191DF011197CB01022E02C0969590
:101DB00087950A94E2F7817081958527842385278A
:101DC0008C932F5F3F4F2330310559F7089580934F
:101DD000EE057093F0056093EF0580911606843050
:101DE000F9F48093E9008FEF9091E800815095FD20
:101DF00006C095ED9A95F1F700008111F5CF80911D
:101E0000E80085FF0DC050E040E063E070E08EEE3A
:101E100095E00E94A6048091E8008E778093E80008
:101E20000895BC0184E00E94E70E0895BC0183E0A0
:101E30000E94E70E08959C0184E08093E9009FEFE3
:101E40008091E800915085FD06C085ED8A95F1F7F7
:101E500000009111F5CF8091E80085FF0CC050E0A3
:101E600040E066E070E0C9010E94A6048091E800AD
:101E70008E778093E8000895CF93DF93EC018091F3
:101E800013018823B1F18091EC0587FF32C060E235
:101E900084E08093E9008FEF9091E800815095FDF8
:101EA00006C095ED9A95F1F700008111F5CF80916C
:101EB000E80085FF1BC08091130170E050E040E016
:101EC000811104C050E040E068E070E0CE010E9463
:101ED000A6048091E8008E778093E80080E2FE01FE
:101EE000A4EFB5E001900D928A95E1F7DF91CF91D3
:101EF000089568E081E0CDCF81E08093E00080E24A
:101F00008093D8001092C9008FE19EE40197F1F709
:101F100000C0000087E090EBDC01809357069093AF
:101F20005806A0935906B0935A0688E19CE00FB674
:101F3000F894A895809360000FBE90936000FFCF47
:101F4000CF93DF93C7EFD2E060E0CE010E94802DF7
:101F50002196C11584E0D807B9F7DF91CF91089594
:101F60001F93CF93DF93122F8430E0F46630D0F4C8
:101F70004F30C0F4C42FD0E0CC0FDD1F9EE1699F2D
:101F8000C00DD11D112494EB899FC00DD11D1124CA
:101F9000632FCE0187960E94802D612FCE018896F7
:101FA0000E94802DDF91CF911F910895AF92BF9233
:101FB000CF92DF92EF92FF921F93CF93DF938CEC3F
:101FC000C82E84E0D82ED0E07601C0E014C0F50120
:101FD00025913491412F6C2F8D2F0E94B00F82E0FC
:101FE000A80EB11C1F5F1F3091F78EE1E80EF11CA7
:101FF000CF5FC63019F0570110E0E9CFDF5F84EB07
:10200000C80ED11CD43001F7DF91CF911F91FF9002
:10201000EF90DF90CF90BF90AF900895CF93C82FEF
:102020006FEF811162E283E290E00E94802D6FEFFA
:10203000C11168E084E290E00E94802D6FEFC11131
:1020400064E085E290E00E94802DCF91089580E0C9
:102050000E940E1060E086E290E00E94802D0E94B7
:10206000D60F0E94A00F81E00E940E1008950F93DA
:102070001F93CF93DF93843030F5663020F54F30D7
:1020800010F5C42FD0E0CC0FDD1F2EE1629FC00DF4
:10209000D11D112434EB839FC00DD11D1124CE011D
:1020A00087960E94622D082F10E0102F0027CE0186
:1020B00088960E94622D9801282BC901DF91CF914B
:1020C0001F910F91089590E080E0F8CF462F843063
:1020D00040F4763030F46F3020F4672F0E943710D0
:1020E000089590E080E00895CF92DF92FF920F93E1
:1020F0001F93CF93DF936C010091560680917B0371
:10210000082BC7E0D0E010E0FC2EC8010C2E02C066
:10211000959587950A94E2F780FD0CC02197A0F76A
:10212000F12C8F2DDF91CF911F910F91FF90DF90B8
:10213000CF900895B6018C2F0E9466100E94DD0C8E
:10214000019761F3EECFCF93DF93EC010E947410FF
:10215000BE010E9466100E94DD0CDF91CF910895B0
:10216000FC01808191810E94A31092959F7096300E
:1021700091F058F4925F9F70923058F4803F19F0BC
:1021800030F4883E30F481E008959A5FF4CF843FC4
:10219000D1F380E00895883EB0F3813FD1F7F3CFCB
:1021A00083E290E00E94622D823289F484E290E022
:1021B0000E94622D883059F485E290E00E94622DE1
:1021C00091E0843009F090E0892F8170089580E0DB
:1021D000FCCFCF9384E090E00E94622DC82F82E272
:1021E00090E00E94622D982F8C2FCF910895EF924E
:1021F000FF920F931F93CF93DF93062F10E00B55A1
:102200001A4FF8019081992321F1E82EEE0CF0E9A4
:102210006F9FE0011124CB50DC4F84E2F82EF09246
:10222000E103E2EEF3E0DE018D91819383E0E23F92
:10223000F807D1F724E630E041E150E061EE73E0C9
:102240008E2D0E942E2CE0E1FE0E6096F4EBFF1224
:10225000E6CFF8011082CDB7DEB7E6E00C948B2C08
:1022600060E084E70E94F71061E086E70E94F710C3
:1022700062E085E70E94F7100895E1EEF3E06083E5
:10228000418324E630E042E050E0BF01880F0E9425
:102290002E2C0895EF92FF920F931F93CF93DF930D
:1022A000E82E062F10E002521A4FF8018081882391
:1022B00081F0F2E16F9FE0011124C855DA4FF12C53
:1022C00049916F2D8E2D0E943D11F39482E1F812F9
:1022D000F7CFF8011082CDB7DEB7E6E00C948B2C77
:1022E000CF93DF93C82F4BE06DEF0E943D1140E08C
:1022F0006AE08C2F0E943D118FE39CE90197F1F772
:1023000000C0000040E060E08C2F0E943D1140E0E2
:1023100061E08C2F0E943D1140E066E08C2F0E940E
:102320003D1140E06DEF8C2F0E943D11D0E040E068
:102330006D2F8C2F0E943D11DF5FD231C1F740E03D
:102340006D2F8C2F0E943D11DF5FD432C1F740E02A
:102350006D2F8C2F0E943D11DF5FD43BC1F74BE006
:102360006DEF8C2F0E943D1141E06AE08C2F0E949E
:102370003D1140E06DEF8C2F0E943D11DF91CF9118
:102380000895A4E0B0E0E7ECF1E10C94702CF62E97
:10239000042F122F8635910570F5880F991F880F2D
:1023A000991FBC016C587C4F44E050E0CE0101966F
:1023B0000E94332D89818370EA81282F30E040E923
:1023C000849FC00111248B509C4FE80FF92FF11D01
:1023D000B497F082EB81E80FF92FF11DB4970083D9
:1023E000EC81E80FF92FF11DB49710832B553A4F6C
:1023F00081E0F90180832496E5E00C948C2CFF9217
:102400000F931F93CF93DF93182F062FF42ED0E056
:10241000C0E02F2D402F612FCE010E94C1112196C7
:10242000C635D105B1F7CDB7DEB7E5E00C948C2CFD
:10243000A4E0B0E0EEE1F2E10C94672C0E948B2B5B
:1024400084E70E94701186E70E94701185E70E9460
:10245000701104E713E052E1752E68E0C62ED12C0E
:10246000EE24E394F12C6624639444E050E0B80138
:10247000CE0101960E94332D4A8150E0CA01849713
:102480002B81622F6452770B4B012C81E22FE45297
:10249000FF0B5F012981237030E0FC0197FD379627
:1024A00043E0F595E7954A95E1F7729EA001739E8A
:1024B000500D112448555A4FE40FF52FF11DB60168
:1024C0000E949A2CA70101C0440F8A95EAF78081E7
:1024D000842B8083F40197FC379693E0F595E7957C
:1024E0009A95E1F7729EC001739E900D1124885554
:1024F0009A4FE80FF92FF11DC401B6010E949A2CE2
:10250000A70101C0440F8A95EAF78081842B80835C
:10251000F501B7FC379683E0F595E7958A95E1F7E5
:10252000729EC001739E900D112488559A4FE80F3A
:10253000F92FF11DC501B6010E949A2CA70101C017
:10254000440F8A95EAF78081842B808322523A4F88
:10255000F90160820C5F1F4FF4E00C3C1F0709F08B
:1025600084CF60E084E70E944A1161E086E70E9420
:102570004A1162E085E70E944A112496EEE00C942D
:10258000832CB0E0A0E0E7ECF2E10C946E2C8C011F
:10259000FC01EF57FD4F8081682349F1D09026065A
:1025A000D0912706C0912506EC2EF12C0E94232DF8
:1025B000282FC7018C549F4F68E671E00E949A2C27
:1025C0008E199F0997FD0396959587959595879503
:1025D00023706C2F289F600D11247D2D8D2F0E945C
:1025E000E408462F282F672FC8010E94DD07CDB7CA
:1025F000DEB7E7E00C948A2CB0E0A0E0E2E0F3E183
:102600000C946B2C182F80911101811323C0909191
:10261000240693702091100130E081E09217130698
:1026200009F480E0817080931601809129069091D1
:102630001501981739F08093150140E060E080E0C3
:102640000E94DA07123160F4E12FF0E0E75FF14D0C
:102650000C94AE2C81E0E6CF80911601811102C06E
:10266000C0E0B0C040E060E080E00E94DA07F8CF50
:10267000C091140182E1C89FC02D112402E10C0F0A
:10268000F02E073510F0F6E5FF2E609125067091CB
:102690002606809127060E94E408E62ED72EC82E33
:1026A000D0E0CF1528F0C1E0063508F48BC0D8CFB4
:1026B000FE01EF57FD4F808190911501892331F084
:1026C0002C2D4E2D6D2DCE010E94DD072196E9CFD8
:1026D000C091140182E1C89FC02D112402E10C0FAA
:1026E000F02E073510F0E6E5FE2EE0902506D0919D
:1026F0002606D09027066091280666956695669511
:1027000080912006909121060E94DA080E948B0891
:10271000805887FD8195880F382F2D2D329F312DC0
:102720001124832F6E2D7D2F0E94E408E62ED72ED4
:10273000C82ED0E0CF1508F0B6CFFE01EF57FD4F01
:10274000808190911501892331F02C2D4E2D6D2D16
:10275000CE010E94DD072196EDCF8EE598E00E9424
:10276000B50A04C088ED97E00E94220BC82F2AC04A
:102770008FEC97E0F9CF86EC97E0F6CF88EB97E007
:10278000EECFC091140182E1C89FC02D112472E1E7
:10279000F72EFC0EEF2C86E58F1510F466E5E62E7D
:1027A00060912806669580912006909121060E94EE
:1027B000DA08D82ED0E0CE15E8F0C1E025E52F15D7
:1027C00008F44ECF809114018F5F80931401C111E2
:1027D0000CC082E08093120180911601811105C026
:1027E000111103C083E080931201CDB7DEB7EAE098
:1027F0000C94872CFE01EF57FD4F808190911501BD
:10280000892311F1CE01880F991F85589E4FFC0135
:10281000E55AFF4F20812152330B865A9F4FFC010E
:1028200040814C55550B609125067091260680918C
:1028300027060D2D0E947A080E94E408462F282FB3
:10284000672FCE010E94DD072196B5CF8AE498E07C
:1028500086CFC091140182E1C89FC02D112442E1AE
:10286000F42EFC0ECF2C36E53F1510F436E5C32EC2
:1028700060912806669566958091200690912106C4
:102880000E94DA08D82E80E48D0D0E948B0890E813
:10289000B92EB80E8D2D0E948B0820E8A22EA80E0E
:1028A000D0E0CC1530F0C1E0E5E5EF1508F08ACFB7
:1028B000D7CEFE01EF57FD4F8081909115018923FE
:1028C000A1F0609125067091260680912706ED2CD7
:1028D0000C2F2A2D4B2D0E94E0070E94E408462F62
:1028E000282F672FCE010E94DD072196DACFC091F5
:1028F0001601C1111EC06091280620E1620F08F484
:102900006FEF80912006909121060E94DA086AE01C
:1029100070E00E944F2C892B09F0A2CE0E94232D3B
:1029200066E570E00E949A2C609115010E94C11228
:1029300049CFC091140182E1C89FC02D112402E14A
:102940000C0F802F073508F086E5D0E0E82EF12C3B
:10295000CE15DF050CF0A7CE60911501CE010E94C7
:10296000C1122196F5CF81EB97E00E94420AFECE7C
:102970008BEA97E0FACF80912A0621E0382F321BAC
:1029800008F430E0832F62E977E00E947809EECE08
:1029900080912A0621E0382F321B08F430E0832F83
:1029A00067E577E0F2CF80912A0621E0382F321BCD
:1029B00008F430E0832F6FE377E0E7CF69E277E058
:1029C00080E0E3CF46E050E06CE170E084E296E026
:1029D0000E94702D1092E00308958F929F92AF9203
:1029E000BF92CF92DF92EF92FF921F93CF93DF932C
:1029F0008091DB039091DC03A091DD03B091DE03B5
:102A00002FB7F8948090E8059090E905A090EA052A
:102A1000B090EB052FBF75016401C81AD90AEA0A04
:102A2000FB0A2FB7F8944091E8055091E9056091B1
:102A3000EA057091EB052FBF4093DB035093DC0355
:102A40006093DD037093DE031091B203E2EBF3E0D9
:102A5000C12FD0E00197AF4FBF4F88199909AA093C
:102A6000BB091D1327C0C093B2038091DF03C0E0F0
:102A7000811108C080912406C82FC37019F0C82F97
:102A8000C695C695809112018130F1F1882329F114
:102A9000823009F44AC0833009F452C0DF91CF91EB
:102AA0001F91FF90EF90DF90CF90BF90AF909F90DD
:102AB0008F900895218D328D4901B12CA12C88155C
:102AC0009905AA05BB0520F4C150DF5F3296C9CF36
:102AD0002C0D3D1D328F218FF8CF109214014093A1
:102AE000200650932106609322067093230689E204
:102AF000E2EBF3E0AAE2B6E001900D928A95E1F7ED
:102B000081E080931201CACF8C2F0E94FC12CC234B
:102B100029F20E94690681FFC1CF2FEF4FEF6FEFBF
:102B20008CE290E00E94DD07B9CFC0931101809143
:102B300024068370809310010E94301183E0E1CF5E
:102B40008091E00381110E94E2144091200650918F
:102B5000210660912206709123062FB7F894809188
:102B6000E8059091E905A091EA05B091EB052FBF2A
:102B7000841B950BA60BB70B4097A105B10508F474
:102B80008DCF109212018ACFE4E2F6E085E18083D6
:102B90008091170190911801A0911901818392836E
:102BA000A3838FE784838FEF85830E94E2140895C7
:102BB0008091790390917803892B8093DA02909128
:102BC0007A039923A1F0892B8093DA028091130173
:102BD0008823E1F18091EC0587FF38C08EE1ECEDB0
:102BE000F2E090E08150A0F591110E94650E40E264
:102BF00050E068E573E08AED92E00E943C2D892B5D
:102C000021F180E2EAEDF2E0A8E5B3E001900D9257
:102C10008A95E1F7E091E305F091E4053097A9F09A
:102C200080911301882359F08091EC0587FF07C03C
:102C30008091DA028093DB0286E08093DA020280E0
:102C4000F381E02D8AED92E00995089586E0C7CFE3
:102C50002191222339F29F5FC5CF882321F00E9462
:102C60006B0E0E94D8150895882339F0909179034E
:102C7000982B909379030E94D815089590E080E0F6
:102C80000E946A2D883E9E4F19F40E94D01008952C
:102C900080E0089568EE7EEF90E080E00E949E2D37
:102CA00060E082E090E00E94802D60E083E090E0B0
:102CB0000E94802D10927B0360E084E090E00E94EF
:102CC000802D64E082E290E00E94802D60E085E04B
:102CD00090E00E94802D60E086E090E00E94802DD0
:102CE0006FEF87E090E00E94802D40E050E0BA0155
:102CF00088E090E00E94922D60E08DE090E00E94DC
:102D0000802D40E050E0BA0188E190E00E94922DD1
:102D100060E087E190E00E94802D40E050E0BA0141
:102D20008CE190E00E94922D70E060E080E290E003
:102D30000E949E2D40E050E0BA0188E190E00E94A0
:102D4000922D80E00E940E100E94271040E050E07B
:102D5000BA018FE090E00E94922D40E050E0BA016D
:102D600083E190E00E94922D08951F920F920FB67A
:102D70000F9211242F933F934F935F936F937F9301
:102D80008F939F93AF93BF93EF93FF938091E10055
:102D900082FF09C08091E20082FF05C08091E100BE
:102DA0008B7F8093E1008091DA0080FF24C08091C6
:102DB000D80080FF20C08091DA008E7F8093DA00F7
:102DC0008091D90080FF9DC080E189BD82E189BDED
:102DD00009B400FEFDCF81E0809316068091F105D5
:102DE000811109C00E9456040E9421058091E200D1
:102DF00084608093E2008091E10080FF17C08091A1
:102E0000E20080FF13C08091E2008E7F8093E20099
:102E10008091E20080618093E2008091D80080621E
:102E20008093D80019BC85E0809316068091E1005C
:102E300084FF2BC08091E20084FF27C080E189BD20
:102E400082E189BD89B5982F917080FFFBCF809179
:102E5000D8008F7D8093D8008091E1008F7E809391
:102E6000E1008091E2008F7E8093E2008091E20099
:102E700081608093E20080911706882309F447C09F
:102E800084E080931606809116068091E10083FF0E
:102E900027C08091E20083FF23C08091E100877FFB
:102EA0008093E10082E080931606109217068091CD
:102EB000E1008E7F8093E1008091E2008E7F80931D
:102EC000E2008091E20080618093E20042E060E0F5
:102ED00080E00E94EF048091F00088608093F00011
:102EE000FF91EF91BF91AF919F918F917F916F91E2
:102EF0005F914F913F912F910F900FBE0F901F90B8
:102F0000189519BC109216061092F10574CF809195
:102F1000E30087FD93E090931606B5CF78941F9257
:102F20001FB61F9211248F939F93AF93BF938091ED
:102F3000E8059091E905A091EA05B091EB050196AD
:102F4000A11DB11D8093E8059093E905A093EA05C2
:102F5000B093EB05BF91AF919F918F911F901FBED2
:102F60001F9018959C014FB7F8948091E8059091B7
:102F7000E905A091EA05B091EB054FBF821B930BC9
:102F800008952FB7F8948091E8059091E905A091F4
:102F9000EA05B091EB052FBF08950E94C1179C016F
:102FA0009091AE038091AF03982B21F03093AB0347
:102FB0002093AA039091B0038091B103982B21F044
:102FC0003093A9032093A803E091E305F091E40571
:102FD000309749F082E08093AC030480F581E02DC6
:102FE0008CEA93E00995089590E080E00E945306F2
:102FF00090E080E00E943D06109278030E94D81570
:1030000086E0ECEAF3E0DF011D928A95E9F7109281
:10301000A6031092A5031092A7030E94CD1708954E
:10302000809356060E94F417089580915606982FB3
:103030009670963021F488600E9410180895877F5A
:10304000FBCF21E030E001C0220F8A95EAF72095FE
:103050008091560682230E9410180895909157037C
:103060008095892380935703282F277091F4282F68
:10307000082E000C330B9217130659F09091ED05B2
:1030800092FF07C08595859585950E94211810921D
:1030900057030895CF93C091ED05C2FB992790F98E
:1030A000981791F080FBC2F9C093ED056091EC0593
:1030B00084E090E00E94802D6C2F82E290E00E94DC
:1030C000802D82E00E942E18CF91089521E030E0FB
:1030D00001C0220F8A95EAF780915606822B0E9442
:1030E0001018089580937B030E94F417089510929E
:1030F000790380911301ECEDF2E0882361F0809177
:10310000EC0587FF08C08EE1DF011D928A95E9F783
:103110000E94F417089586E0F7CFAAE2B0E0E3E951
:10312000F8E10C94722C88E196E02091F100DC012A
:103130002D93CD01B6E080329B07B9F78091190637
:10314000833009F472C0B8F4813009F449C0823088
:1031500009F4B3C08091E80083FF8BC28091180608
:10316000909119069A3008F084C2E92FF0E0E55EEC
:10317000F14D0C94AE2C8A3009F48EC08B3009F4DA
:1031800071C0893039F780911806813219F7809122
:103190001C0690911D06009711F00297D9F68091B8
:1031A000E800877F8093E8008091E80082FF38C0C4
:1031B0009091F3008091F200029731F48091F10038
:1031C000813011F0863021F48091F1008093F30575
:1031D0008091E8008B778093E8000E94D004BACFFA
:1031E00080911806813A09F0B5CF8091E800877F79
:1031F0008093E80080911C0690911D06892B61F454
:1032000060E284EF95E070E00E947C058091E80028
:103210008B778093E8009ECF60E090E080E0F3CF72
:10322000809116068111C0CF95CF80911806813A02
:1032300009F090CF80911C0690911D06892B09F012
:1032400089CF8091E800877F8093E8008091E80033
:1032500080FFFCCF809113018093F1008091E80002
:103260008E77B9CF80911806813209F073CF8091A3
:103270001C0690911D06892B09F06CCF8091E80007
:10328000877F8093E8000E94D00480911A06809383
:1032900013010E9477185ECF80911806813209F0E1
:1032A00059CF8091E800877F8093E8000E94D00486
:1032B00080911B068093F2054DCF80911806813ACC
:1032C00009F048CF8091E800877F8093E8008091E3
:1032D000E80080FFFCCF8091F205BECF803899F0E6
:1032E000823809F0C6C180911C068F70873008F0C3
:1032F000C0C18093E9008091EB0085FB882780F9AD
:103300001092E90006C08091140690911506911163
:1033100082609091E800977F9093E8008093F1009D
:103320001092F1008091E8008E779FC1882309F404
:103330008DC1823009F09DC180911A06811190C122
:1033400080911C068F702FEF280F263008F091C156
:103350008093E9002091EB0020FF82C1933031F48B
:103360008091EB0080628093EB007AC19091EB003A
:1033700090619093EB0021E030E001C0220F8A952C
:10338000EAF72093EA001092EA008091EB0088604F
:10339000EACF81116EC110911A061F778091E30068
:1033A0008078812B8093E3008091E800877F809371
:1033B000E8000E94D0048091E80080FFFCCF80915B
:1033C000E30080688093E30082E0111183E0809342
:1033D00016064FC18058823008F04BC120911A0662
:1033E00030911B062C3DE3E03E07A1F583E08A8384
:1033F0008AE289834FB7F894DE01139620E03EE01D
:1034000051E2E32FF0E050935700E49120FF03C016
:10341000E295EF703F5FEF708E2F90E0EA30C0F0E2
:10342000C7968D939D932F5F243159F74FBF80919D
:10343000E800877F8093E8006AE270E0CE010196A1
:103440000E947C058091E8008B778093E80011C191
:10345000C096E7CF80911C0690911D06432F5527FB
:103460004330510509F44AC078F54130510509F45B
:103470007AC08BE590E0ECE9F7E04230510509F0C5
:10348000F8C02091E800277F2093E80020911E06D5
:1034900030911F068217930708F49C0140E0211524
:1034A000310509F065C0411163C08091E80082FDDB
:1034B000C9CF80911606882329F2853019F28091B0
:1034C000E80083FFF2CFBECF4132510509F43CC082
:1034D0004232510509F0CDC08330910508F0C9C0D2
:1034E000FC01EE0FFF1FE159FE4F0190F081E02D2E
:1034F00084599E4FDC018C9190E01AC03327213013
:103500003105D1F02115310561F02230310509F086
:10351000B0C0E9E0F8E0E4918E2F90E0E9E0F8E057
:1035200007C0E3E3F8E0E4918E2F90E0E3E3F8E0F6
:10353000009709F49EC0A5CFE3E2F8E0E4918E2F56
:1035400090E0E3E2F8E0F4CF8330910508F091C019
:10355000880F991FFC01EB58FE4F0190F081E02D80
:1035600089E090E08ECF82E190E0E7EFF7E089CF4D
:1035700080911606882309F465CF853009F462CF5F
:103580008091E80083FD5ECF8091E80082FD8DCFC1
:103590008091E80080FF83CF9091F3008091F2004A
:1035A0002115310519F08830910550F041E0089758
:1035B00009F040E08091E8008E778093E8006FCFBB
:1035C00044914093F1003196215031090196E8CFA2
:1035D000803809F04EC08091E800877F8093E80032
:1035E000809117068093F1009DCE811142C0109109
:1035F0001A061230F0F58091E800877F8093E8008A
:10360000109317060E94D004112311F084E005C026
:103610008091E30087FDFACF81E08093160642E0B7
:1036200061EC81E00E94EF0442E261EC84E00E94E0
:10363000EF0442E261EC82E00E94EF0442E260ECBF
:1036400083E00E94EF048091160613C080911A0651
:10365000813079F481E0933009F080E080931506A1
:103660001092E9008091E800877F8093E8000E9433
:10367000D0048091E80083FF0AC08091E800877F32
:103680008093E8008091EB0080628093EB00AA9623
:10369000E3E00C948E2C1F920F920FB60F92112420
:1036A0002F933F934F935F936F937F938F939F934A
:1036B000AF93BF93CF93DF93EF93FF93D091E90044
:1036C000DF708091EC00C82FC17080FDC0E81092BF
:1036D000E9008091F000877F8093F00078940E9449
:1036E0008D181092E9008091F00088608093F000BE
:1036F000CD2BCF70C093E900FF91EF91DF91CF9177
:10370000BF91AF919F918F917F916F915F914F91F9
:103710003F912F910F900FBE0F901F9018950E9410
:1037200077182FEF84E39CE0215080409040E1F730
:1037300000C0000088E19CE00FB6F894A895809343
:1037400060000FBE90936000FFCF882391F19CEF43
:10375000980F913A40F4682F8AED92E00E94DE05BE
:103760000E94D815089590E2980F983050F4877011
:1037700091E001C0990F8A95EAF7892F0E946B0E9C
:10378000EFCF9BE5980F933028F490E080E00E9403
:103790005306089598E5980F973128F490E080E05B
:1037A0000E943D060895803F20F00E946C0B0E940D
:1037B000CD170895CF93C82F8823D1F18CEF8C0FAC
:1037C000813AC0F580911301882311F18091EC05B5
:1037D00087FF1EC0EC2FE695E695E695F0E0E652F1
:1037E000FD4F828190E04C2F477021E030E002C015
:1037F000220F331F4A95E2F782239323892B89F006
:103800006C2F8AED92E00E94DE050E94D81509C057
:10381000ECEDF2E08191C81799F382E0E23EF807FF
:10382000C9F76C2F8AED92E00E9408060E94D81515
:10383000CF91089580E28C0F883068F4C77021E042
:1038400030E001C0220FCA95EAF780917903822BFC
:1038500080937903EBCFEBE5EC0FE33040F4F0E03D
:10386000E65EFE4F808190E00E945306E1CFE8E5DE
:10387000EC0FE73150F4F0E0EE0FFF1FE35EFE4F78
:10388000808191810E943D06D3CFC03F88F28C2F6A
:103890000E94270C0E94CD17CBCF1F93CF93DF93AD
:1038A000182FD0E0C0E0893311F4C0E5D0E0812FBB
:1038B0000E94DA1B209739F4812F0E94A51BDF910B
:1038C000CF911F9108958FE99FE00197F1F700C014
:1038D00000002197EFCF0F931F93CF93DF93C62F55
:1038E000D42F022FFC0182818823A9F06093550612
:1038F0000E94C1179093540680935306C77081E0CD
:1039000001C0880FCA95EAF70E943416DF91CF9163
:103910001F910F91089580915506681332C08091D0
:103920005306909154060E94B217883C910548F5C1
:1039300010E21D0FCD17B9F080E28C0F883040F4F3
:10394000C77081E001C0880FCA95EAF70E942D1662
:10395000183048F481E09D2F977001C0880F9A9528
:10396000EAF70E943416802F0E944D1C183070F622
:10397000D77081E001C0880FDA95EAF70E942D1612
:10398000C5CFC77081E001C0880FCA95EAF7F6CFAE
:10399000A5E0B0E0EEECFCE10C94642C8C01FC01A1
:1039A00083819481892B31F08081918189238F3F9C
:1039B00009F08DC52596E1E10C94802C0E947410CD
:1039C000F82E682F89819A810E94B00E69817A81D0
:1039D0008F2D0E9466107C01F8018281882309F4F2
:1039E0003CC5970122513F452031310508F062C5A1
:1039F0008FEF93E00E94622D811128C0FEEEEF0E42
:103A000057EF852E52E0952EE11032C01C821B82AA
:103A1000442443944AE0342E74018FEFE81AF80AE4
:103A2000C4010E94622D89831A82882379F09FEF56
:103A3000980F933058F58A83498292E0890E911C41
:103A4000C7010E94622D8B83811121C08091570391
:103A5000877009F4AFCFF8018281882309F4AACFD7
:103A60008091ED0582FFA6CF82E00E942E18A2CFA2
:103A7000811424E0920651F3C4010E94622D811149
:103A800001C0EA943FEF831A930ABECF4701FE01BB
:103A900031967F01F7012081222309F4BDCF213027
:103AA00009F047C091818281913031F4F2E0EF0E4C
:103AB000F11C0E944D1C07C0923049F422E0E20E36
:103AC000F11C0E94DA1B3FEFE31AF30AE3CF9330B5
:103AD00031F432E0E30EF11C0E94A51BF4CF9430C8
:103AE00021F08FEFE81AF80AEECF92E0E90EF11C10
:103AF00030E020E0B7016F5F7F4FF70141818053D5
:103B0000990B8A30910550F021503109E0F28FE98C
:103B10009FE00197F1F700C00000F6CF329EF00160
:103B2000339EF00D11249C012E0F3F1F842F7B012B
:103B3000E1CFE22FF0E0EC50FE4F5490822F8695BB
:103B40008695869590E0FC01EC51FE4F64902770BD
:103B5000712C022E02C0759467940A94E2F7E1E09A
:103B60006E227724FC01EC52FE4FA490B12C022E61
:103B700002C0B594A7940A94E2F7F1E0AF22BB2407
:103B8000FC01EC53FE4FC490D12C02C0D594C794D5
:103B90002A95E2F721E0C222DD246114710419F0B4
:103BA00081EE0E94DA1BA114B10419F086EE0E9486
:103BB000DA1B852D0E944D1CA114B10419F086EE6C
:103BC0000E94A51B6114710419F081EE0E94A51BCF
:103BD000C114D10409F477CF8CE26BCF81E00E944D
:103BE00066180E94151832CF81E00E942118F9CF83
:103BF00082E0FBCF95EFE9169CE5F90609F46CC06D
:103C000008F466C027E245EE66EEF6EFEF16FCE537
:103C1000FF0609F44BC4882309F46AC410925506C0
:103C200023E0E2162DE5F20608F05DC03AEFE31658
:103C30003CE5F30630F4C70182509C45449708F0F8
:103C40005EC00E94E9109093ED058093EC05E1E1E0
:103C5000EE16ECE5FE0609F438C108F0A6C029E02E
:103C6000E2162CE5F20609F41EC108F06FC085E0EB
:103C7000E8168CE5F80609F40AC108F058C0E3E03C
:103C8000EE16ECE5FE0609F4F8C008F0FCC08091E1
:103C9000EC05816022E0E2162CE5F20609F4F0C0A2
:103CA0006091EC05F090ED0584E090E00E94802D9D
:103CB0006F2D82E290E00E94802D0E947718C6CE80
:103CC00027E245EE65EEF2C326E241EE60EEEEC37A
:103CD00027E245EE64EEEAC326E241EE62EEE6C379
:103CE00028E241E0EFCF81E6E8168DE5F80609F419
:103CF000A8CF95EAE9169DE5F90609F4A2CF36E1C9
:103D0000E3163CE5F30609F071C4809179038A7AE1
:103D100091E009F490E09093FA0269E2811165E381
:103D20008AED92E00E9408060E94D8158FCE8091FD
:103D3000EC05806237E0E3163CE5F30609F4A0C029
:103D400008F4ADC08091EC0580649AC08091EC05C8
:103D50008B7F9DE0E9169CE5F90609F491C0B0F46B
:103D60008091EC058E7FFBE0EF16FCE5FF0609F481
:103D700087C08091EC058C602CE0E2162CE5F20601
:103D800008F47EC08091EC058D7F7AC08091EC05AF
:103D90008F7E3FE0E3163CE5F30609F471C008F4BA
:103DA00088C08091EC058F7D6BC09DEFE9169CE586
:103DB000F90609F486C078F5F5E1EF16FCE5FF0693
:103DC00009F491C0A0F48091EC05837F33E1E31600
:103DD0003CE5F30609F454C008F47BC00E94771850
:103DE0009091EC05892F97FB87F9805849C09BEF8C
:103DF000E9169CE5F90609F44EC008F05EC0809112
:103E0000ED058160FAEFEF16FCE5FF0609F048CFFB
:103E10008093ED0545CF21E0E2162DE5F20609F489
:103E20006EC0B8F48FEFE8168CE5F80609F457C0B9
:103E30008091ED058360E1149DE5F90648F38091DA
:103E4000ED05982F909591708E7F892B90FB81F9CD
:103E5000DFCFE1E6EE16EDE5FE0609F456C0F5EA21
:103E6000EF16FDE5FF0609F457C022E0E2162DE546
:103E7000F20609F015CF60E043C08091EC05826046
:103E80008093EC050DCF8091EC058460F9CF809193
:103E9000EC058860F5CF8091ED058260B9CF809107
:103EA000EC058061EDCF0E9477188091EC05806869
:103EB000E7CF8091EC05877FE3CF8091ED058E7F82
:103EC000A7CF8091ED058D7FA3CF8091EC058F7BEF
:103ED000D7CF0E9477188091EC058F77D1CF809152
:103EE000ED058C7F95CF8091EC0582FB992790F9A9
:103EF00021E0922790FB82F990FB83F9C1CF61E02A
:103F00008EE090E00E94802DCBCE9091EC05892F21
:103F10008F7E94FF8061B4CF9091EC05892F8E7FC6
:103F200090FF8160ADCF8091FA0269E2811165E373
:103F30008AED92E00E94DE05F7CE42E157E06DE1A6
:103F400077E00E94760682CD4DE157E062E177E0AE
:103F5000F8CF43EE56E06EEE76E0F3CF4EEE56E04D
:103F600063EE76E0EECF47EC56E065ED76E0E9CF24
:103F700045ED56E067EC76E0E4CF49EB56E06BEABE
:103F800076E0DFCF4CE756E06AE876E0DACF4AE841
:103F900056E06CE776E0D5CF61E081E00E94F9065B
:103FA00055CD61E085E0FACF0E9477188FEF94E35A
:103FB000ECE081509040E040E1F700C000000E943A
:103FC0007C0F8091ED0582FB882780F991E089279D
:103FD0000E944A18F8018281E080F180882309F468
:103FE00045C0C7010E947410D82E682FC7010E94D7
:103FF000B00EB7018D2D0E9466100E94DD0C7C0171
:10400000882EF801D280B580B2943FE0B32280912F
:1040100057038770C1F0AD2CDD20B1F08F2D807F6C
:10402000803421F080E28E0D883068F08091ED05BB
:1040300082FF09C082E00E942E188091570387708A
:10404000AA24A3948111A12C9F2C92942FE0922258
:10405000FBE0F91508F479C0E92DF0E0EB5DF14DD6
:104060000C94AE2C81E0B4CF80E0B2CFC7010E94A7
:104070007C0ED82EBECF2F2D2F70C22E8F2D807F7D
:1040800019F0C29490EFC922DD20B9F0CC2069F07C
:1040900080E28E0D883010F0811009C08091790384
:1040A000C82AC09279030E94D8158E2D4CC08091E9
:1040B0007803C82AC0927803F6CF8E2D0E94A51BE4
:1040C000CC2009F442C080E28E0D883010F08110BF
:1040D00004C08C2D0E946B0E06C0C09480917803A2
:1040E000C822C09278030E94D8152FC03F2D3F7080
:1040F000C32E8F2D807F803219F0C29480EFC822AA
:10410000882089F081E0881609F468C0DD2009F470
:1041100072C0BB2009F468C0F801858180FFC5CF5B
:104120008F70858361C02091ED0522FD35C0DD20B3
:1041300069F1CC2039F080917903C82AC0927903C3
:104140000E94D81580E00E94DA1B292D2850330BDD
:104150002430310510F40E946906AA2009F42ACC03
:104160008091570380FD26CCF801128285958595B4
:1041700085950E946618C8010E94C81C809157034B
:104180008595859585950E94211814CC80E00E9424
:10419000A51BCC20D1F29DCFDD2099F090917A0320
:1041A000892F8C29B11003C00E943416CECFE1E0D4
:1041B000BE12FACF22FFC9CF981739F280937A0343
:1041C000C4CFB11006C00E94650E8C2D0E942D1622
:1041D000BCCFF1E0BF1609F4B8CFF5CFDD2031F048
:1041E00025E02B1508F4B1CF8C2DDECF34E03B1544
:1041F00008F4ABCFEACFBB2041F3F9E38F1209C03B
:104200002FEF37EE83E0215030408040E1F700C0CF
:1042100000008E2D0E94A51B98CF8F2D8695869528
:10422000837061F0813009F090CFC7019370D11095
:1042300002C090E080E00E943D0687CFC7019370E6
:10424000D11002C090E080E00E9453067ECF8E2DF8
:10425000DD2029F00E94270C0E94CD1776CF0E9406
:104260006C0BFACF8F2D837091F5D1106ECF4E2D40
:10427000429546954770440F440F8E2D8F70042E43
:1042800001C0880F0A94EAF72E2D2071E4FE07C0C2
:104290002FE030E001C0220F4A95EAF720953F2D2C
:1042A000369536953370323069F050F440917B0387
:1042B000313029F0822B84230E94721846CF842B40
:1042C000822BFACF282B80917B038227F5CF86950E
:1042D000DD2011F08F2D8170882309F436CF4E2D0B
:1042E000429546954770440F440F8E2D8F70042ED3
:1042F00001C0880F0A94EAF72E2D2071E4FE07C052
:104300002FE030E001C0220F4A95EAF720953F2DBB
:10431000369536953370323069F050F44091560638
:10432000313029F0822B84230E9410180ECF842B69
:10433000822BFACF282B809156068227F5CF9F2D0E
:104340009F70F92EDD2029F0892F0E9466188E2D8E
:104350002BCF8E2D0E942D168F2D0E942118F5CE69
:104360008E2DE2EF8E16B1F1E81570F0F0EF8F169A
:10437000D1F021EF821691F0DD2009F45EC0B1107A
:1043800094CE8F2D8F712AC033EF831651F194EFA5
:104390008912F2CF8091ED0582FD2FC08F2D8F7194
:1043A000DD20D9F21BC0DD2081F0E4E0EB1508F43C
:1043B000CCCE2F2D2F7181E090E001C0880F2A957F
:1043C000EAF7909156068927AFCFF5E0FB1508F480
:1043D000BCCEEFCF8F2D8F71D110BFCF0E9466184A
:1043E000B4CE80E0DD2009F49FCF9F2D9F7181E046
:1043F00001C0880F9A95EAF797CFDD2099F02F2D0D
:104400002F71F22E822F0E9466188091ED0582FF97
:1044100007C038E0F39EC0011124836080935703E6
:104420008F2DDCCF81E00E942E1881E08B1508F0E3
:104430008CCE82E00E942E1888CEBB2059F08933A2
:1044400009F0E7CE9FEFE7EEF3E09150E040F04057
:10445000E1F7DDCE8F2D8F7180CFF0E1EF16FFE514
:10446000FF0609F4C1CB21E1E2162FE5F20609F4BB
:10447000BFCB93EFE9169CE5F90609F425CC08F0CB
:10448000B9CBF8EDEF16FCE5FF0609F419CC29EDE0
:10449000E2162CE5F20609F423CC37EDE3163CE5F1
:1044A000F30609F0B8CB26E241EE61EEC8010E94A6
:1044B0006B1CCCCA30E1E3163FE5F30609F48ECB62
:1044C00091E1E9169FE5F906A1F682E088CB85E047
:1044D000DE01119601900D928A95E1F7F801228193
:1044E00089819A8121116ACA0E947C0EF82E6ECAB7
:1044F000F6E1EF16FCE5FF0609F415CD809179038E
:1045000082722AECE2162CE5F20609F436CDE0F5CB
:1045100095ECE9169CE5F90609F41BCDE0F4F3EC03
:10452000EF16FCE5FF0609F408CD08F00DCD32ECDE
:10453000E3163CE5F30609F04DCD8091240691E0A9
:10454000892780932406109212018091E0038160F4
:104550008093E0037BCA97ECE9169CE5F90609F421
:1045600002CD08F4FBCCF8ECEF16FCE5FF0609F4ED
:10457000FFCC4BEA56E069EB76E029ECE2162CE53D
:10458000F20609F4DECC26CD3FECE3163CE5F3065B
:1045900009F407CDB8F4ECECEE16ECE5FE0609F4F0
:1045A000F6CC08F4EFCC2DECE2162CE5F20609F47B
:1045B000F3CC61E082E03EECE3163CE5F30609F45F
:1045C000EDCC08CD86EDE8168CE5F80648F461E000
:1045D00088E091EDE9169CE5F90608F4DFCC36CACF
:1045E000EDE5EE16FE0609F431CAF4CCFAE5EF1655
:1045F000FDE5FF0609F436CD78F4E1143CE5F30659
:1046000009F4D2CC8EEDE8168CE5F80609F0E2CC80
:104610000E944A160E948F1B9CE5E9169DE5F9064B
:1046200009F4CFCC08F420CDF7EAEF16FDE5FF063C
:1046300089F3D0CC1F93CF93DF9380912403807FA5
:1046400009F049C080912103882309F444C0809176
:104650005603D091250360911F0370912003A09110
:104660002203B0912303C62FC72316E0D81799F170
:1046700090E0109711F0CF3F19F401968770F6CFB4
:10468000189F9001199F300D1124F901EA5DFC4F2C
:1046900041814713F2CF40814613EFCF4281411150
:1046A000ECCF438154814A1B5B0B483C510528F7F2
:1046B000809124038F70806180932403F901E55D6C
:1046C000FC4F80818F70806180838FE193E00E9436
:1046D000C81C0E94720EDF91CF911F910895A1E135
:1046E000B0E0E5E7F3E20C946B2C8C0185E0F80177
:1046F000DE011D9601900D928A95E1F7F801E280A6
:104700008FE1A82E83E0B82E6091220370912303DD
:104710006115710509F426C190911F034091200392
:10472000892F84238F3F09F41DC120813181C380EB
:10473000D480F0902103F601E61BF70BFF2009F46B
:10474000DCC080912403582F507FE83CF10508F02D
:104750009FC051116BC0FE2C431314C0921312C0A2
:10476000E11010C08F70806180932403C5010E9406
:10477000C81C80912403F80185838F2D6196EAE09F
:104780000C94872CC114D10429F0822F83238F3FEE
:1047900009F003C180E0F82FF170DF2E80FF3CC0EC
:1047A000809156034091250356E0841315C02D8750
:1047B0003E878D859E850E94A310292F22952F70FC
:1047C0002230F0F0243018F59F70F1F0F801958157
:1047D000907FD1F4D12C1EC090E0589FF001599FDA
:1047E000F00D1124EA5DFC4F6181361306C0608133
:1047F000261303C06281E6120FC001968770D5CFE1
:104800009F7011F0882331F3805E883018F3C8015F
:104810000E94C81CFD2CB1CFEE2009F4AECF8091D0
:104820002403816080932403F12CA7CF431306C097
:10483000921304C0F801EE2009F479C0C8010E9467
:10484000B010882309F1EE20F9F080912403803222
:1048500070F020911F033091200338872F83198631
:10486000DB86CA868C87CE0107960E94C81C86E02C
:10487000F801AFE1B3E001900D928A95E1F70E9453
:104880001A23FF24F39479CFC8010E94C81CF9CFE2
:1048900051110AC08FE193E00E94C81C86E0F50127
:1048A00011928A95E9F7C0CF43130FC092130DC040
:1048B000E1100BC0F8018583C8010E94C81C86E086
:1048C000F50111928A95E9F758CFC8010E94B010FE
:1048D0008823D1F2EE20C1F280912403803238F295
:1048E00020911F03309120033A8329831B82DD82AC
:1048F000CC828E83CE010196B8CFE83CF105F8F664
:10490000FE2CEE2009F243131FC092131DC08091AC
:10491000240380FD10C0982F907F69F0F8018583F3
:10492000903F31F0982F907F905F8F70892B858317
:10493000C8010E94C81C86E0F801AFE1B3E0019015
:104940000D928A95E1F719CFC8010E94B01081112C
:104950008ECF80912403816080932403C8010E943C
:10496000C81C0BCFEE2009F48FCFC8010E94B010F5
:10497000F82E882309F488CF86E0F801AFE1B3E090
:1049800001900D928A95E1F780911F039091200389
:104990000E94A3100E941A23F0CE81E08E25FBCE48
:1049A000A7E1B0E0E6EDF4E20C94722C4B8B5C8B4B
:1049B0006D8B7E8B8F8B6111109278031A8A198A06
:1049C00085E0FE017396DE011D9601900D928A9599
:1049D000E1F786E0FE013D96DE01179601900D920B
:1049E0008A95E1F7CE0107960E946F23811112C0CC
:1049F00086E0FE013796DE01119601900D928A95B0
:104A0000E1F78A859B85892B29F088859F818923F9
:104A10008F3F81F516E0809156039091250389130D
:104A200017C06796E3E00C948E2C96E0929FD0011D
:104A3000939FB00D1124AA5DBC4FFE0131960190E9
:104A40000D929A95E1F7809325030E94720EE2CFB2
:104A5000819FC00111248A5D9C4F0E946F2388238F
:104A600001F38091560390E0019687709927809317
:104A70005603D1CF2091250330E0C90101968770FC
:104A80009927409156034817190679F60E9477181E
:104A9000109225031092560386E0EFE1F3E0DF0168
:104AA0001D928A95E9F7B6CFACE0B0E0EAE5F5E211
:104AB0000C94692C8E010F5F1F4F8CE0F80111924E
:104AC0008A95E9F79BE4E92E91E0F92E6801AA2482
:104AD000A394B12CF70181917F018F3F09F446C067
:104AE000F894E82FE295EF70F0E021A18F70A50116
:104AF00002C0440F551F8A95E2F7CA01922F982BE6
:104B000091A392A18095892382A3789400C0E1E5C6
:104B1000F1E021E030E0912C812C41914F3F09F4EC
:104B200089C0A42FA295AF70B0E090968C9190E0D0
:104B30004F7002C0959587954A95E2F780FD7AC03F
:104B4000C901882A992A220F331F51E0E036F50760
:104B500021F7F701319780818F3F11F00E94830C7C
:104B600080EA8A95F1F7F60191828082F2E0CF0E19
:104B7000D11C41E5E41641E0F40609F0ABCF4CE06E
:104B800050E0B8018FE793E00E943C2DFF24F3949E
:104B9000009709F4F12C892B09F44FC08CE0F8013F
:104BA000AFE7B3E001900D928A95E1F781E0809341
:104BB0007E030E94C11790937D0380937C038091B4
:104BC0007C0390917D030E94B2170397D0F18091EE
:104BD0007F039091800390939A038093990380912F
:104BE00081039091820390939C0380939B03809117
:104BF00083039091840390939E0380939D038091FF
:104C00008503909186039093A00380939F038091E6
:104C10008703909188039093A2038093A1038091CE
:104C2000890390918A039093A4038093A303109225
:104C30007E0307C090E080E084CF80917E038111E5
:104C4000BECF8F2D2C96ECE00C94852C1F921FB6B6
:104C50001F9211248F939F93AF93BF938091E70589
:104C6000811113C08091E8059091E905A091EA05B2
:104C7000B091EB054196A11DB11D8093E80590937D
:104C8000E905A093EA05B093EB05BF91AF919F9121
:104C90008F911F901FBE1F901895CDB7DEB7AA97B2
:104CA0000FB6F894DEBF0FBECDBF85B7806885BF55
:104CB00085B7806885BF84B7877F84BF0FB6F894B7
:104CC000A8958091600088618093600010926000D8
:104CD0000FBE80E890E00FB6F89480936100909347
:104CE00061000FBE81E89CE09093D9028093D802C6
:104CF0000E9456040E9421058091E2008460809306
:104D0000E2007894809116068823A1F01091E900C2
:104D10001F709091EC00892F817090FD80E8182B16
:104D20001092E9008091E80083FD0E948D181F70A9
:104D30001093E90082E084BD93E095BD9AEF97BDA2
:104D400080936E000E94D010811102C00E94271033
:104D50000BE411E0D8018D918D018F3F11F00E947D
:104D6000830CB1E001351B07A9F701E511E0F8015B
:104D700081918F018F3F11F00E94830CF1E000368A
:104D80001F07A9F78CE0E9E9F3E0DF01282F1D9266
:104D90002A95E9F7EFE7F3E0DF011D928A95E9F73D
:104DA0000E943E16811102C00E944A1682E090E0E5
:104DB0000E94622D80938B030E94E9109093ED0571
:104DC0008093EC050E945425EFEBFDE53197F1F758
:104DD00000C000000E9454258091990380FF08C004
:104DE0006FEF7FEF90E080E00E949E2D0E947C0F8D
:104DF00083E090E00E94622D0E9472180E941812B7
:104E000010922A068FEF9FEF9093440680934306FB
:104E100090934606809345069093480680934706F4
:104E200090934A068093490690934C0680934B06D4
:104E300090934E0680934D069093500680934F06B4
:104E400090935206809351061092B2039093CC0334
:104E50008093CB039093CE038093CD039093D003A4
:104E60008093CF039093D2038093D1039093D40384
:104E70008093D3039093D6038093D5039093D80364
:104E80008093D7039093DA038093D9030E943E1650
:104E9000811104C00E944A160E94C41546E050E0E9
:104EA0006CE170E084E296E00E94522D1092E003E3
:104EB000809124068C7F11F40E94C41584E091E057
:104EC0009093E4058093E30538E1632E712C40E470
:104ED000342EBB24B394442443948091160623E0DB
:104EE000F22E00E112E1853009F4FAC10E94542546
:104EF000882359F08FB7F8944091E8055091E9055F
:104F00006091EA057091EB058FBF99E9C92E93E096
:104F1000D92EACE8B3E0F60110E000E0602FE1909C
:104F2000F1902D913D912E153F0509F404C2A12C5D
:104F300088248394912C2E253F25A90148215921AD
:104F4000452B09F4F2C1A9A26AA3E820F92081E067
:104F5000E114F10409F480E08BA30E94C117816081
:104F6000782F9DA38CA349A15AA16BA18DA10E946A
:104F7000D024F801EE0FFF1FE457FC4F8081918190
:104F80008826992691828082EF2871F08FE0809F99
:104F9000F001819FF00D1124E558FE4FEA0DF11D3F
:104FA00080818F3F09F0A8C1A12C0A2D10E08091CB
:104FB000B203800F912F911D09976CF188E090E06A
:104FC0007C01E01AF10AB8016D547C4FA70183EB14
:104FD00093E00E94492DB80165547C4FA7018BEBEB
:104FE00093E00E94492DA701440F551FB801660F99
:104FF000771F65537C4F8BEC93E00E94492DB801DD
:105000006D537C4FA70183EC93E00E94492D88E00B
:105010008A198093B2038091B20390E0A52DB0E08D
:105020009D01220F331F2B523E4FAA0FBB1FBD0104
:105030006A527E4F41E0480F9A1508F461C180938F
:10504000B2030E94ED1486E0ECEAF3E0DE01119673
:1050500001900D928A95E1F71092AE031092AF0382
:105060001092B0031092B1038B819C81892B09F4BB
:105070004AC08091AA039091AB030E94B2179C0191
:105080009091A603992309F441C325313105D8F144
:105090009F3F19F09F5F9093A6031B81112359F046
:1050A0000E94070C9FEF11160CF491E0899F802D50
:1050B00011248093AE031C81112359F00E94070C28
:1050C0009FEF11160CF491E0899F802D112480939D
:1050D000AF033091AE033323B1F02091AF0322230D
:1050E00091F045EB3403C0011124992309F43AC12E
:1050F0009093AE0345EB240390011124332309F46C
:1051000034C13093AF038D819E81892B09F44AC04D
:105110008091A8039091A9030E94B2179C019091DD
:10512000A503992309F4EDC221353105D8F19F3F3C
:1051300019F09F5F9093A5031D81112359F00E94E0
:10514000E50B9FEF11160CF491E0899F802D11243F
:105150008093B0031E81112359F00E94E50B9FEF4D
:1051600011160CF491E0899F802D11248093B103D6
:105170003091B0033323B1F02091B103222391F099
:1051800045EB3403C0011124992309F4F1C0909335
:10519000B00345EB240390011124332309F4EBC041
:1051A0003093B10346E050E0BE016F5F7F4F8CEA61
:1051B00093E00E943C2D892B61F48091AE03909185
:1051C000AF03892B9091B003892B9091B103892B68
:1051D00011F00E94CD1786E0FE013196ACEAB3E0F3
:1051E00001900D928A95E1F70E94690690919803CB
:1051F00089138093980380911606843009F06DCE50
:1052000083E08093E9008091E80082FF66CE809180
:10521000E80090E085FF06C00E947504882309F429
:10522000ADC091E08091E8008B778093E8009923EE
:1052300009F453CEE981E150E33108F01FC1F0E0F9
:10524000EF5CF14D0C94AE2C80911606843009F47D
:1052500036C00E94ED148091DF0381110DC00E94C1
:10526000FC1210921101809124068370809310012A
:105270000E943011F09212014092DF031092E70574
:105280000FB6F894A895609260000FBE309260004F
:1052900083B7817F846083BF83B7816083BF789445
:1052A000889583B78E7F83BF0FB6F894A8958091B9
:1052B0006000886180936000109260000FBE809152
:1052C0001506882369F00E945425E9E9F3E08191ED
:1052D0009191892B09F0F6C123E0E53AF207B9F77D
:1052E00080911606853009F4AFCF0E9477180E948E
:1052F00069061092DF03FACD582EAA24A39455CE46
:1053000090E0FC01EE54FC4FD9015C915183DB012C
:105310005C915187518A880F991FFC01EE54FC4F14
:10532000128E118E91E0842F85CEA394880C991C47
:105330004FE0A41202CE0F5F1F4F0630110509F097
:10534000EDCD8FEF8EA38FA318A60E94C1178160A9
:10535000782F9AA789A74EA15FA168A58AA50E9468
:10536000D0246FCEB092AE03C5CEB092AF03CBCEF9
:10537000B092B0030ECFB092B10314CF00E210E0B0
:10538000CE0101967C018091E80085FD0AC08091E4
:10539000E8008B778093E8000E947504882399F3D6
:1053A00040CF8091F100D7018D937D01015011090B
:1053B00051F737CF1A8289E0C7C08A81823009F459
:1053C00097C18330D9F1813009F058C02FB7F894D4
:1053D0006091E8057091E9058091EA059091EB05EF
:1053E0002FBF0E94B42C6B837C838D839E8380911E
:1053F0001606843009F071CD1091E9001F7090916C
:10540000EC00892F817090FD80E8182B82E080935A
:10541000E9008091E80080FF0DC050E040E060E2CC
:1054200070E0CE0101960E94A6048091E8008E777C
:105430008093E8001F701093E9004FCDFE01319674
:10544000D6018C9111969C91B2E0CB0ED11C928327
:105450008383329625EAC21623E0D20689F7C7CFA6
:105460008A81823059F46B817C818D819E810E947A
:10547000B42C86E290E00E94802DB9CF8FEF898313
:10548000B6CF4C816B818A810E943710982789277B
:1054900098279E838D83ABCF2D813E813227232792
:1054A00032274C816B818A810E94B00FA0CF0E946D
:1054B000D60F9DCF8A818138C9F068F4803809F011
:1054C00096CF8091250620E04B816091260690E0E2
:1054D0000E9498068CCF823819F1833809F087CF63
:1054E0008B8120E0409127066C81F1CF60E08B81B9
:1054F0000E94F9069B8180912406911109C0982F82
:10550000937011F0109212018C7F809324066FCF5C
:10551000982F937011F4109212018C7F8160F5CF57
:10552000EB818FE7E43020F4F0E0E05AFE4F808119
:10553000809328065CCF8A818138A1F038F48038C6
:1055400009F055CF809127068B8351CF823879F0AF
:10555000833809F04CCF809125068B8380912606F5
:105560008C8345CF8091240686958695EDCF8091DA
:105570002806873230F08F3530F08E3930F083E0F6
:10558000E3CF80E0E1CF81E0DFCF82E0DDCF0E949A
:10559000E2142DCF80E18A832ACFBA820CCF0A8110
:1055A0001B81102701271027CE0101967C01CC809A
:1055B000DC01AC0DB11D6D01C80189509D4FCE14A9
:1055C000DF0409F414CF0930B1E01B0750F40E9446
:1055D000622DF70184830F5F1F4FBFEFEB1AFB0AA9
:1055E000EBCFD70114961C92F6CF0A811B811027AE
:1055F00001271027FE0131966F01EC80E00EF12E9D
:10560000F11CC80189509D4F0E151F0509F4EFCEFE
:105610000930F1E01F0728F4D60114966C910E941E
:10562000802DBFEFCB1ADB0A0F5F1F4FEACF0E941E
:10563000A00FDDCE84E0AFCF0A811B8110270127A8
:105640001027FE0131967F01CC80CF018C0D911D7A
:105650006C01C8018796CE14DF0409F4C8CE003D62
:10566000A2E01A0750F40E94622DF70184830F5FB5
:105670001F4FBFEFEB1AFB0AECCFD70114961C9219
:10568000F6CF0A811B81102701271027FE013196D2
:105690006F01EC80E00EF12EF11CC80187960E150B
:1056A0001F0509F4A4CE003DF2E01F0728F4D6013F
:1056B00014966C910E94802DBFEFCB1ADB0A0F5F0E
:1056C0001F4FEBCF09BD19BD09B400FEFDCF80917E
:1056D000D8008F7D8093D8008091E0008260809315
:1056E000E0008091E00081FDFCCF0E947718F8CDAA
:1056F00086E290E00E94622D1B821C821D828E83B6
:1057000076CE2B30310508F014CD4CCD2B30310541
:1057100008F0C0CCF8CC1092B9008CE08093B800AF
:105720000895B0E0A0E0E7E9FBE20C946A2CB82E03
:10573000EB010E94C1176C01EE24E394F12CC431FB
:10574000D10560F025E0E22EF12CCF3FDC0731F0EF
:10575000CE0164E170E00E944F2C7B0184EAA82E08
:1057600094E8992E1092BC00A092BC000E94C11730
:105770008C018091BC0087FF0DC08091B900887FAB
:10578000883001F18091B900887F8031D9F00FEF26
:105790001FEF09C00E94C117801B910B8E159F053A
:1057A00040F30EEF1FEFCF3FDC07E1F2C6010E948E
:1057B000B2178C179D07B0F2C801CDB7DEB7EBE08A
:1057C0000C94862CB092BB009092BC000E94C11732
:1057D0008C018091BC0087FF0AC08091B900887F4E
:1057E000883111F0803499F610E000E0E5CF0E9496
:1057F000C117801B910B8E159F0558F3D2CF0F93C5
:105800001F93CF93DF93EB018093BB0084E88093D9
:10581000BC000E94C1178C018091BC0087FF11C0A1
:105820002091B900287F81E090E0283211F490E0C7
:1058300080E0919581959109DF91CF911F910F9112
:105840000895CF3FDC0741F30E94C117801B910BE5
:105850008C179D0708F38EEF9FEFEECFB0E0A0E02E
:10586000E4E3FCE20C946D2C6B018A017901B9012F
:105870000E94912BE6010C0D1D1DC017D10711F0E0
:1058800097FF08C024E92093BC00CDB7DEB7E8E05D
:105890000C94892CB70189910E94FF2BEECFAA1B93
:1058A000BB1B51E107C0AA1FBB1FA617B70710F00B
:1058B000A61BB70B881F991F5A95A9F7809590953D
:1058C000BC01CD0108952F923F924F925F926F924B
:1058D0007F928F929F92AF92BF92CF92DF92EF9280
:1058E000FF920F931F93CF93DF93CDB7DEB7CA1B01
:1058F000DB0B0FB6F894DEBF0FBECDBF09942A882C
:10590000398848885F846E847D848C849B84AA84D3
:10591000B984C884DF80EE80FD800C811B81AA8160
:10592000B981CE0FD11D0FB6F894DEBF0FBECDBF2B
:10593000ED01089597FB072E16F4009407D077FD2C
:1059400009D00E944F2C07FC05D03EF4909581951C
:105950009F4F0895709561957F4F0895EE0FFF1F3B
:105960000590F491E02D09946927962769277827F7
:10597000872778270895CF92DF92EF92FF92CF93F7
:10598000DF93CDB7DEB72A970FB6F894DEBF0FBE10
:10599000CDBF89879A87A985BA852D913D914D9173
:1059A0005C9129833A834B835C83232B242B252B07
:1059B00041F424E239ED4BE557E029833A834B83E8
:1059C0005C8369817A818B819C812DE133EF41E099
:1059D00050E00E94A42D69017A01A7EAB1E49B017D
:1059E000AC010E94C32D69837A838B839C83ACEEC8
:1059F000B4EFA70196010E94D12D9B01AC018981D2
:105A00009A81AB81BC81820F931FA41FB51FB7FF82
:105A100003C00197A109B048E985FA858083918385
:105A2000A283B3839F772A960FB6F894DEBF0FBE8A
:105A3000CDBFDF91CF91FF90EF90DF90CF90089591
:105A40000E94BB2C089580E091E00E94BB2C089539
:105A5000B0E0A0E08093000190930101A0930201C7
:105A6000B09303010895FB01DC0102C005900D9283
:105A700041505040D8F70895FB01DC0104C08D91DE
:105A80000190801921F441505040C8F7881B990BB0
:105A90000895FB01DC0102C001900D92415050407D
:105AA000D8F70895DC01CB01FC01F999FECF06C0BF
:105AB000F2BDE1BDF89A319600B40D9241505040CC
:105AC000B8F70895F999FECF92BD81BDF89A99274C
:105AD00080B50895A8E1B0E042E050E00C94542D68
:105AE000DC01A40FB51F4150504048F0CB01840F9A
:105AF000951F2E910E94812D41505040D0F708955E
:105B0000262FF999FECF92BD81BDF89A019700B476
:105B1000021639F01FBA20BD0FB6F894FA9AF99A16
:105B20000FBE08950396272F0E94812D0E94802D7D
:105B3000252F0E94812D242F0C94812D0196272F33
:105B40000E94812D0C94802D052E97FB1EF400944D
:105B50000E94BB2D57FD07D00E94D62D07FC03D015
:105B60004EF40C94BB2D50954095309521953F4FA8
:105B70004F4F5F4F089590958095709561957F4F39
:105B80008F4F9F4F08950E94F82DA59F900DB49FB1
:105B9000900DA49F800D911D11240895B7FF0C94C2
:105BA000C32D0E94C32D821B930B0895A1E21A2ED0
:105BB000AA1BBB1BFD010DC0AA1FBB1FEE1FFF1FB1
:105BC000A217B307E407F50720F0A21BB30BE40B01
:105BD000F50B661F771F881F991F1A9469F7609548
:105BE0007095809590959B01AC01BD01CF01089502
:105BF000A29FB001B39FC001A39F700D811D11240E
:105C0000911DB29F700D811D1124911D0895F8946E
:105C1000FFCF2C1338136813AD13B213B813BB1393
:105C2000BE13C113261429147714B314B814BB146B
:105C3000C814D314DE146E199619391B9619391B22
:105C4000C919EA19391BE81AF51A3B203B207620BE
:105C500076200D212721A520A52032219F21B021CA
:105C6000B021DA29DD29302A412A4C2A572A5A2A1A
:105C70009B2AC72A3E2A3E2ACA2ACD2ACF2AF52A9B
:085C8000172B1A2B1C2B412BE2
:105C880001000000DB053C0F1B0F160F110FDA0592
:105C9800FFFF030100FF0000FFC8818283E200E9E3
:105CA80000EA00B500B600B700CD008301CC008A39
:105CB80001920194012102230224022502260227CF
:105CC800022A02B300B4006F007000F7F6F5F4F191
:105CD800F03031323337929395949697343536664F
:105CE8000F3F7FBD003131295A1B750A4022B68407
:105CF800016201AC00AE07C707E707000102030411
:105D080005060708090A0B0C0D0E0F1011121314C3
:105D1800FF15161718191A1B1C1D1E1F20212223D8
:105D28002425262728292A2B2C2D2E2F30313233B3
:105D38003435363738393A3B3C3D3E3F40414243A3
:105D48004445464748FF494A4BFF4C4D4E4FFF508C
:105D58005152535455000010001E002B00380048C3
:105D68000055006300700080008D009A00A700BEF7
:105D780000D800000D100D200C310E421052146690
:105D8800147610860E960CA70DB80DC50DD80D000B
:105D98001A0F1A1F172F183F1C4E1E691E781C88D1
:105DA800189817A81AB81AC51AD21AE01A00250F97
:105DB800251E212D233C254B285C2B6C287C258A0D
:105DC800239921A825B825CB25E02500300E301DC4
:105DD8002C2B2E393048325C3570327E308D2E9B1C
:105DE8002CA930B830D230003A0E3A223A3D3D5311
:105DF8004064407A3D953AAA3AB83AC53AD23AE070
:105E08003A04040404040404040404040404040414
:105E1800040404040404040404040404040404043A
:105E2800040404040404040404040404040404042A
:105E3800040404040404040404040404040404041A
:105E4800040404040404040404010404040404040D
:085E580004040404010101002F
:00000001FF
